:020000040800F2
:10000000300400209F3A0000DF380000DF38000095
:10001000DF380000DF380000DF380000000000009B
:100020000000000000000000000000000D3900008A
:100030000D390000000000000D390000B738000045
:100040000D3900000D3900000D3900000D39000098
:100050000D3900000D390000353900005D39000010
:1000600085390000AD390000D53900000D39000098
:100070000D3900000D3900000D3900000D39000068
:100080000D3900000D390000FB3900000D3900006A
:100090000D3900000D3900000D3900000D39000048
:1000A0000D3900000D3900000D3900000D39000038
:1000B000233A00004B3A0000733A00000D3900006B
:1000C0000D3900000D3900000D3900000D39000018
:1000D0000D3900000D3900000D3900000D39000008
:1000E0000D3900000D3900000D3900000D390000F8
:1000F0000D3900000D3900000D3900000D390000E8
:100100000D3900000D3900000D3900000D390000D7
:100110000D3900000D3900000D3900000D390000C7
:100120000D3900000D3900000D3900000D390000B7
:100130000D3900000D3900000D3900000D390000A7
:100140000D3900000D3900000D3900000D39000097
:100150000D3900000D3900000D3900000D39000087
:100160000D3900000D3900000D3900000D39000077
:100170000D3900000D3900000D3900000D39000067
:100180000D3900000D390000AE010000FFFF1F2DEA
:100190002D2D204D6563726973702D5374656C6CE1
:1001A0006172697320322E352E32202D2D2DC6011D
:1001B00000004200043264757000386847F8046D2E
:1001C000043F38607047D801000062000532647255
:1001D0006F70043740CF7047F601000044000532CD
:1001E0007377617007CF043F386047F8046D043FB0
:1001F0003A600E0070470A020000620004326E6925
:10020000700007CF043F38607047240200004400AC
:1002100005326F766572B86847F8046D043F386040
:10022000FE68704748020000440005327475636B35
:1002300007CF043F386047F8046D043F3A60043F3D
:100240003960043F386070476A020000460004329B
:10025000726F74003868B9683A69B86039613A6099
:1002600079687E60FE68F96070478C020000460085
:1002700005322D726F743868B9683A69386139602F
:10028000BA60F968FE607E6879607047A00200007D
:10029000200003323E7201CF01B440B440CF70471A
:1002A000B802000020000332723E47F8046D40BCE3
:1002B00001BC043F38607047D002000020000332C8
:1002C000724047F8046D019E47F8046D009E704728
:1002D000E2020000200006327264726F700002B009
:1002E0007047FA02000042000364322F3868F107B9
:1002F000761040080843386070470E030000620023
:100300000364322A38680018764138607047280341
:10031000000042000464736872003868F1077608D0
:1003200040080843386070473E03000062000464E0
:1003300073686C0038680018764138607047500365
:1003400000004200046461627300002E07D470470D
:100350006E030000420007646E656761746538686B
:100360000021C043F64301304E4138607047860398
:100370000000640002642D0007CF121AB1410E0084
:10038000043F3A6070479C030000640002642B0045
:1003900007CF12184E41043F3A607047AE03000089
:1003A000610003733E6447F8046DF6177047C2039B
:1003B0000000620003756D2A3868A0FB06063860ED
:1003C0007047D60300006200026D2A00386880FB87
:1003D0000606386070471404000044000375642A60
:1003E00007CF564341437618010C130C5943761836
:1003F000010C80B292B25143434350430022C918CA
:1004000052411204B6180A04090C80184E41043FE8
:1004100038607047A604000044000475646D2A002B
:1004200010B5002447F8046D7E6847F8046D3E69F6
:10043000FFF7C2FF310040CF300040CF47F8046DD6
:100440003E6847F8046DFE6803B4FFF7B5FF03BCD0
:10045000330040CF320040CF47F8046D3E6847F884
:10046000046D3E690FB4FFF7A7FF0FBC92196341FB
:1004700040CF89196241634140CF47F8046D7E68DF
:1004800047F8046DFE680FB4FFF796FF0FBC921992
:10049000634140CF89196241634140CF1E003A60F9
:1004A0007960B86010BDC80400004300022A2F0024
:1004B00000B540B440CFFFF789FF47F8046D40BC5A
:1004C00000F04CF8043700BDEA0400004300052AA0
:1004D0002F6D6F6400B540B440CFFFF777FF47F84A
:1004E000046D40BC00F03AF800BD0C05000043006C
:1004F00003752A2F00B540B440CFFFF75DFF47F8E2
:10050000046D40BC00F01BF8043700BD300500004E
:10051000430006752A2F6D6F640000B540B440CFCC
:10052000FFF74AFF47F8046D40BC00F008F800BD33
:1005300050050000430006756D2F6D6F640000B517
:1005400047F8046D002600F019F840CF043700BDCD
:100550006E0500004300056D2F6D6F6400B547F810
:10056000046DF61700F032F840CF043700BDC00527
:10057000000044000675642F6D6F640030B40023E2
:1005800000227968B86835003C684026400049413F
:1005900052415B41AB4202D804D3A24202D3121BA8
:1005A000AB410130013EF1D10E0038607B60BA6092
:1005B00030BC704730B400237A68B9680020E2E7A5
:1005C00036060000440005642F6D6F6400B5F01717
:1005D00019D0FFF7C4FEFFF705FEF0170CD0FFF7A8
:1005E000BEFEFFF7FFFDFFF7C9FFFFF7FBFDFFF7BB
:1005F000B6FEFFF7F7FD00BDFFF7F4FDFFF7BEFF06
:10060000FFF7ADFE00BDFFF7EDFDF0170ED0FFF7D1
:10061000A6FEFFF7E7FDFFF7B1FFFFF7A0FEFFF72C
:10062000E1FDFFF79CFEFFF7DDFD00BDFFF7DAFD02
:10063000FFF7A4FF00BD4C060000440002642F0039
:1006400000B5FFF7C3FFFFF7DCFD00BD9406000017
:10065000440002662A0000B5F0170DD0FFF77FFEB8
:10066000FFF7C0FDF0170DD0FFF779FEFFF7D8FEBA
:1006700040CF01CF386000BDFFF7B4FDF017F5D0D3
:10068000FFF76DFEFFF7CCFE40CF01CF3860FFF7DC
:1006900066FE00BDE0060000440002662F0000B5C3
:1006A000F0170ED0FFF75BFEFFF79CFDF0170ED0A2
:1006B000FFF755FEFFF796FDFFF77CFFFFF7A1FD63
:1006C00000BDFFF78FFDF017F4D0FFF748FEFFF7EE
:1006D00089FDFFF76FFFFFF742FEFFF792FD00BDB8
:1006E000F406000020000232210006CF3160726063
:1006F00040CF704708070000200002324000043F4E
:1007000070683860366870471C0700004400036456
:10071000753C07CF121AB141B6417047300700004F
:1007200044000364753E07CF801A8E41B64170477E
:1007300046070000440002643C0007CF121AB14192
:100740000CDB0026704762070000440002643E0094
:1007500007CF801A8E4101DB002670470026F64342
:1007600070477207000062000364303C0437F617DC
:1007700070478607000062000364303D01CF0643E6
:10078000013EB6417047A0070000440003643C3EB0
:1007900007CF50404E400643013EB641F6437047F6
:1007A000B8070000440002643D0007CF50404E40AF
:1007B0000643013EB6417047CA070000200003739C
:1007C000704047F8046D3E007047DA0700002000D3
:1007D00003737021370040CF7047EC070000200002
:1007E0000372704047F8046D6E467047FC070000C6
:1007F000200003727021B54640CF70470C080000FE
:1008000061000364757047F8046D70471C080000B0
:1008100061000464726F700040CF704732080000BE
:100820006100043F64757000002E01D047F8046D2C
:1008300070474608000062000473776170003968F1
:100840003E600E007047540800006200036E69703D
:1008500004377047680800006200046F7665720014
:1008600047F8046D7E6870477E08000062000474DB
:1008700075636B0001CF083F7E6038607047940855
:100880000000630003726F7403CF083F78603E601E
:100890000E007047AC0800006300042D726F7400F6
:1008A00003CF083F7E60396006007047BE08000035
:1008B0002000047069636B0057F826607047D60803
:1008C00000000000056465707468BC49C91B47F8E6
:1008D000046D8E107047F208000000000672646517
:1008E0007074680047F8046D6E46B549891B8E1018
:1008F0007047020900002000023E720040B440CF61
:10090000704714090000200002723E0047F8046D91
:1009100040BC70472609000020000272400047F8E2
:10092000046D009E70473609000020000572647255
:100930006F7001B070474A090000200005727069AD
:10094000636BB6006E4436687047600900006E0045
:1009500003616E6401CF064070470640000616F042
:10096000780900006E000362696301CFB04306009E
:1009700070478643000636F08E0900006E00026F55
:10098000720001CF064370470643000656F0A409E3
:1009900000006E0003786F7201CF464070474640FA
:1009A000000696F0B20900006100036E6F74F64312
:1009B0007047C2090000610003636C7AB6FA86F6DC
:1009C0007047D009000061000373687276087047B1
:1009D000DE09000061000373686C76007047EE0961
:1009E0000000610003726F725FEA76067047000ACA
:1009F0000000610003726F6CB61956F10006704773
:100A00001A0A00006C00067273686966740001CFF0
:100A1000F0400600704736080026340A00006C00DB
:100A2000076172736869667401CF304106007047D0
:100A30003610F6174E0A00006C00066C7368696683
:100A4000740001CFB04006007047360000265E0AF1
:100A50000000610002303D00013EB6417047700A5F
:100A60000000610003303C3E013EB641F643704752
:100A70007E0A0000610002303C00F6177047940ABD
:100A80000000600004747275650047F8046D00266C
:100A9000F6437047A80A000060000566616C736544
:100AA00047F8046D00267047BC0A00004200023E71
:100AB0003D0001CFB042EADA00267047D00A0000BC
:100AC0004200023C3D0001CFB042E0DD002670470D
:100AD000E20A00004200013C01CFB042D7DB002611
:100AE0007047F40A00004200013E01CFB042CEDC64
:100AF00000267047080B0000620003753E3D01CFE1
:100B0000861BB641F64370471C0B0000620003755C
:100B10003C3D01CF361AB641F64370472E0B00001C
:100B2000620002753C0001CF861BB6417047400B46
:100B30000000620002753E0001CF361AB6417047D0
:100B4000560B00006B00023C3E0001CF361A013EFE
:100B5000B641F6437047680B00006B00013D01CFC2
:100B6000361A013EB64170477C0B00006200036DEF
:100B7000696E01CFB04200DC06007047900B0000A8
:100B80006200036D617801CFB04200DB0600704760
:100B9000A60B0000620004756D61780001CFB042C1
:100BA00000D306007047C40B0000620004756D6935
:100BB0006E0001CFB04200D806007047300300201D
:100BC00030040020020C00000000046D6F76650008
:100BD00007B5310040CF320040CF00290FD0B242DC
:100BE0000DD006D3013E013A705C50540139FBD15F
:100BF00005E030781070013601320139F9D140CF6B
:100C000007BD240C000000000466696C6C00300015
:100C100040CF310040CF002902D001397054FCD1BF
:100C200040CF7047300C000020000140366870470C
:100C3000480C00006D00012103CF30600E007047AA
:100C400006607047016070476E0C00006D00022B5B
:100C5000210003CF3268121832600E00704702681C
:100C600092190260704702685218026070477C0C4B
:100C7000000020000268400036887047960C000093
:100C80006D000268210003CF30800E00704706809F
:100C9000704701807047BC0C00006D0003682B2179
:100CA00003CF3288121832800E00704702889219E2
:100CB000028070470288521802807047CA0C0000F8
:100CC00020000263400036787047E40C00006D009D
:100CD0000263210003CF30700E007047067070472A
:100CE000017070470A0D00006D0003632B2103CFD4
:100CF0003278121832700E00704702789219027022
:100D000070470278521802707047320D00006D0073
:100D100004626973210003CF3268024332600E001F
:100D20007047026832430260704702680A430260FB
:100D300070475A0D00006D0004626963210003CF03
:100D40003268824332600E0070470268B24302602C
:100D5000704702688A4302607047820D00006D0090
:100D600004786F72210003CF3268424032600E0077
:100D70007047026872400260704702684A40026031
:100D80007047EC0D0000680004626974400001CFF8
:100D90003668064018BF4FF0FF3670474FF4D04218
:100DA00000B5012B0AD147F8046D002600F0C2FF00
:100DB00047F8046D160001F027FB11E002CF013B5C
:100DC00002F0B4FC47F8046D3626164301F01CFB14
:100DD00047F8046D0E0047F8046D002600F0AAFFE6
:100DE00047F8046D8A4E01F0F7F800BD140E0000BC
:100DF0006D0005686269732103CF32880243328037
:100E00000E007047028832430280704702880A430E
:100E1000028070473C0E00006D0005686269632126
:100E200003CF3288824332800E0070470288B2437B
:100E30000280704702888A4302807047640E000077
:100E40006D000568786F722103CF3288424032808E
:100E50000E007047028872400280704702884A4044
:100E600002807047840E0000680005686269744063
:100E700001CF3688064018BF4FF0FF3670474FF459
:100E800008428DE7AC0E00006D00056362697321B6
:100E900003CF3278024332700E007047027832433B
:100EA0000270704702780A4302707047D40E000047
:100EB0006D0005636269632103CF3278824332702B
:100EC0000E0070470278B2430270704702788A437E
:100ED00002707047FC0E00006D000563786F722190
:100EE00003CF3278424032700E0070470278724071
:100EF0000270704702784A40027070471C0F000071
:100F0000680005636269744001CF3678064018BFF7
:100F10004FF0FF3670474FF4F04241E72C0F0000CE
:100F200061000563656C6C2B04367047640F00002C
:100F300061000563656C6C73B600704700F0E4FCFB
:100F40001E466C6173682063616E6E6F742062650B
:100F5000207772697474656E2074776963650A001E
:100F600002F00BBC441000000000083136666C61D2
:100F7000736821003FB54FF00F00304015D000F0EE
:100F8000C3FC223136666C61736821206E6565642E
:100F9000732031362D616C69676E6564206164640D
:100FA000726573730A0002F0E8BB30680130C5D186
:100FB00070680130C2D1B0680130BFD1F068013033
:100FC000BCD14FF00062B618124A134B1360134B9A
:100FD0001360134A4FF00103136008CF04CF02CF10
:100FE00001CF01C602C600F01DF804C608C600F015
:100FF00019F80B4A10684FF0010188431060084A45
:1010000010684FF000410843106040CF3FBD000022
:10101000920D00000840005823016745AB89EFCDD1
:101020001440005807B4294A4FF480311068084230
:10103000FCD14FF0010110680842FCD088431060D9
:1010400007BC7047E410000000000E666C61736816
:10105000706167656572617365000FB5300040CFE0
:101060004FF4804398422FD3194A1A4B13601A4BFE
:1010700013604FF00C01C8404FF0FF0108404FF0E3
:10108000030188404FF002010843144A10604FF4F6
:101090008031084310600D4A13684FF480301840C7
:1010A000FAD10E4A10684FF00041084310600C4A14
:1010B000116802B44FF4C060814311604FF4C05016
:1010C0000143116002BC11600FBD000010400058C8
:1010D0000840005823016745AB89EFCD1440005804
:1010E000004000586611000000000A6572617365D7
:1010F000666C617368004FF4804072B64FF48011E3
:101100004FF6FF72038893421CD047F8046D060027
:1011100047F8046D00F0F8FB1045726173652062BA
:101120006C6F636B20617420200000F055FC00F0B0
:10113000EBFB0C2066726F6D20466C6173680A00D1
:10114000FFF78BFF02308842DCD100F0DDFB124656
:10115000696E69736865642E205265736574202119
:101160000A0002F096FB8211000000000E65726119
:101170007365666C61736866726F6D00300040CF96
:10118000BBE7A4110000000009696E6974666C6118
:10119000736854484FF42071002202700130013905
:1011A000FBD170478C12000000000768666C617309
:1011B000682130B5320040CF500813D300F0A4FBB3
:1011C0001E68666C61736821206E656564732065B6
:1011D00076656E206164647265737365732E0A00B0
:1011E00002F0CBBA4FF480439A4210D200F08CFB4D
:1011F0001943616E6E6F7420777269746520696E31
:10120000746F20636F726520210A02F0B6BA130969
:1012100034482021046824099C4226D01430013926
:10122000F8D1304820210468002C17D0143001393F
:10123000F9D100F069FB21546F6F206D616E792048
:1012400073636174746572656420466C61736820B1
:101250007772697465732E0A02F08FBA1B010360FE
:10126000013941608160C16001610F211140043189
:10127000465240CF0168013101600F221140082918
:1012800003D100F01AF8FFF775FE30BDE812000038
:1012900000000A666C757368666C6173680000B55F
:1012A000104820210268002A03D000F006F8FFF75A
:1012B00061FE14300139F5D100BD47F8046D466870
:1012C00047F8046D866847F8046DC66847F8046DF2
:1012D000066947F8046D0F26F6430268164000229F
:1012E0000260704730040020FE1200006900012BEC
:1012F00001CF3618704736180036000616F1141361
:1013000000006900012D01CF861B7047361A003E90
:101310000006B6F122130000610002312D00013EEB
:10132000704730130000610002312B000136704716
:101330003E130000610002322D00023E70474C1344
:101340000000610002322B00023670475E1300007D
:101350006100066E656761746500764270477013C0
:101360000000610003616273F01736184640704751
:101370008E130000420005752F6D6F6401CF3100A0
:10138000B0FBF6F67143401A043F38607047AC1367
:1013900000004200042F6D6F640001CF310090FB0C
:1013A000F6F67143401A043F38607047C0130000DE
:1013B0004200036D6F6400B5FFF7EFFF40CF00BD43
:1013C000D01300006200012F01CF90FBF6F67047AA
:1013D000E01300006A00012A01CF464370474643EC
:1013E000EE130000610002322A0076007047FC1301
:1013F0000000610002322F007610704710140000C8
:101400006100046576656E00012030403618704733
:1014100028140000810004626173650047F8046DC0
:101420008A4E70470A0000003E1400000000066269
:10143000696E617279008548022101607047541419
:101440000000000007646563696D616C7F480A21D4
:1014500001607047AA1400000000036865787B48AB
:101460001021016070477A494FF0FF000860794908
:101470004FF48040086078494AF2050008607749D7
:101480004FF00100086076494FF0EE400860754962
:101490004FF02300086074494FF48050086073498E
:1014A0004FF00D000860FEE77047C6140000810091
:1014B00009686F6F6B2D656D697447F8046D6C4E2C
:1014C0007047B0150000E2140000810008686F6FDB
:1014D0006B2D6B65790047F8046D664E7047D61525
:1014E00000000015000081000A686F6F6B2D656DAC
:1014F00069743F0047F8046D5F4E704700160000A6
:101500001C150000810009686F6F6B2D6B65793FBA
:1015100047F8046D594E70472E1600003A1500002A
:1015200081000A686F6F6B2D70617573650047F8F5
:10153000046D534E70474238000050150000000003
:1015400004656D6974000FB5494800F026F80FBDB9
:10155000641500000000036B65790FB5454800F085
:101560001CF80FBD76150000000005656D69743F1D
:10157000414800688746881500000000046B6579C3
:101580003F003E48006887469E1500000000057039
:10159000617573653A480068874600688746C415D8
:1015A000000000000B73657269616C2D656D6974D4
:1015B00000B500F025F8002E40CFFAD0314A167061
:1015C00040CF00BDEC15000000000A736572696130
:1015D0006C2D6B65790000B500F029F8002E40CF26
:1015E000FAD047F8046D284A167800BD1C16000092
:1015F00000000C73657269616C2D656D69743F0044
:1016000000B5FFF7C7FF47F8046D00261F480168C3
:101610004FF08000014000D0F64300BD901600005E
:1016200000000B73657269616C2D6B65793F00B5C5
:10163000FFF7B0FF47F8046D0026144801684FF02B
:101640002000014000D0F64300BD0000FCFF032055
:101650004C0000586000005800040048180400487E
:10166000200400480C38014008380140003801408F
:10167000F8FF0320F4FF0320F0FF0320ECFF03201A
:10168000E8FF032028380140243801401C3801407D
:10169000B41600000000076365787065637400B5D8
:1016A000386801B40130386000F00BF801BC0670F6
:1016B00040CF00BD2A17000000000661636365701B
:1016C000740000B502CF01390022FFF746FF300059
:1016D00040CF7F2809D0202819D2092816D00A28FF
:1016E0001FD00D281DD00828EFD1002AEDD000F022
:1016F0000BF903082008002AE7D0885C013A802310
:101700000340E2D040230340F5D0DEE72020B24280
:10171000DBD247F8046D0600FFF715FF013288544D
:10172000D3E7160000F09FF800BD3C170000400012
:101730000374696247F8046D294E70475217000020
:101740008100033E696E47F8046D264E7047000025
:1017500000007817000082000E63757272656E7467
:101760002D736F757263650047F8046D1E4E7047E8
:1017700000000000680000209417000000000973BA
:101780006574736F75726365174802CF06604160B8
:1017900040CF7047B2170000000006736F75726388
:1017A000650047F8046D104E043F70683860366875
:1017B0007047EC17000000000571756572790FB570
:1017C000084800210160FFF7B5FF47F8046D47F8AE
:1017D000046DC826FFF775FFFFF7D6FF0FBD0000A9
:1017E00068000020E4FF0320DCFF03203418000021
:1017F000000007636F6D706172650FB5310040CFF7
:1018000001CF884202CF10D1002810D001380A5CE5
:10181000335C412A02D35B2A38BF2032412B02D3EA
:101820005B2B38BF20339A42EED000260FBD002636
:10183000F6430FBD4818000000000263720000B5B7
:1018400000F062F8010A00BD5A18000000000262B0
:101850006C0047F8046D202670476E1800000000E9
:1018600005737061636547F8046D20266BE68E187A
:1018700000000000067370616365730000B5002E00
:1018800003DDFFF7F0FF013EFBD140CF00BD9E1806
:1018900000005000065B636861725D0005E0B618E9
:1018A0000000000004636861720000B501F0D9FB1C
:1018B00040CF367800BDC61800005000012847F818
:1018C000046D292606E0E01800005000015C47F88E
:1018D000046D002600B501F0CEFB043740CF00BDFB
:1018E000241900003000022E2200AA4800B547F853
:1018F000046D060000F07BFA47F8046D222601F023
:10190000BAFB00F0BBFD00BD0AB447F8046D764693
:10191000013E33780121013319405B181EEB030EA1
:101920000ABC39E04A1900003000026322009A48DC
:10193000DCE747F8046D7646013E33780121013338
:1019400019405B181EEB030E70477419000030003D
:10195000027322009148C9E747F8046D764647F8BC
:10196000046D013E36780121731C19405B181EEB93
:10197000030E70478C190000000005636F756E74CC
:10198000013647F8046D013E36787047A41900000F
:10199000000005637479706500B5FFF7F1FF00F092
:1019A00007F800BDCC1900000000047479706500D0
:1019B00001B501CF002E07D047F8046D0678FFF778
:1019C000C2FD0130013EF7D140CF01BD061A000033
:1019D0000000046865782E0007B5310040CF202054
:1019E0000F22043847F8046D0E00C6401640092E39
:1019F00001D9373600E03036FFF7A5FD0028F0D1D9
:101A0000FFF731FF07BD161A0000000003682E73B0
:101A10001FB5634C0EE0261A0000000003752E73FC
:101A20001FB5604C06E0CA1A00000000022E7300C9
:101A30001FB55D4C5D49C91B8908220A2020292F4A
:101A4000200A2028273E200A202F4343202020332D
:101A500035204343430A385C29295F200A0A544A47
:101A6000106803B40A201060FFF74EFF085374613A
:101A7000636B3A205B0047F8046D0E0001F0D3FC65
:101A8000FFF742FF025D200003BC2736484A106082
:101A900000290AD0474A106806B447F8046D0600CA
:101AA000A04706BC043A0139F5D1FFF72DFF062007
:101AB000544F533A200047F8046D3600A047FFF713
:101AC00023FF04202A3E0A001FBD6A1B00000000FD
:101AD00005776F72647300B5FFF716FF010A00F017
:101AE00034FFFFF711FF09416464726573733A2094
:101AF00047F8046DFFF770FFFFF706FF064C696EAD
:101B00006B3A200047F8046D3668FFF765FFFFF772
:101B1000FBFE07466C6167733A2047F8046DB68890
:101B2000FFF75AFFFFF7F0FE06436F64653A2000A7
:101B3000B01D00F046FF47F8046D0600FFF74CFFAC
:101B4000FFF7E2FE064E616D653A200047F8046D2E
:101B50000636FFF721FFFFF7D7FE010A00F00EFF60
:101B6000300040CFBDD040CF00BDB81B000000000A
:101B700006756E757365640000B500F0D2FF4FF016
:101B8000005001684FF00052914201D24FF480168C
:101B9000761A00BD0819000032190000581900001B
:101BA000D91900001734000027340000300300204A
:101BB000FCFF03202C0300201C1D000000000D3141
:101BC00032626974656E636F64696E670FB5FF2E6C
:101BD00004D847F8046D5FF0FF360FBD16F0FF1014
:101BE000B0420ED14FF6FF710840310C814208D14E
:101BF00016F0FF0656F4805647F8046D5FF0FF3686
:101C00000FBD16F0FF20B0420FD14FF6FF71084014
:101C1000310C814209D1360A16F0FF0656F40056FF
:101C200047F8046D5FF0FF360FBDFF223100114011
:101C3000300A1040884210D1300C104088420CD13C
:101C4000300E1040884208D116F0FF0656F4405678
:101C500047F8046D5FF0FF360FBD30000021013101
:101C6000001850F100007FF07F020240802A05D06A
:101C70001F29F4D347F8046D00260FBD0829F9D3B6
:101C8000060036F0800611F00100C001064311F095
:101C90000E00C002064311F010008005064347F80D
:101CA000046D5FF0FF360FBD47F8046DDFF89C66EA
:101CB0005FF4704110EA0102120116435FF4006103
:101CC00010EA0102D20316435FF4E06110EA010258
:101CD00012011643FF2110EA010216431E43BDE321
:101CE00047F8046DDFF868665FF0704110EA0102A2
:101CF000120B16435FF0006110EA0102520816430E
:101D00005FF0E06110EA0102120B16435FF47F01FD
:101D100010EA0102120C16431E439FE3821D0000CD
:101D200000001072656769737465726C697465721E
:101D3000616C2C000FB5330040CF1B02FF2E05D87D
:101D400056F400561E4300F05FFB0FBDFFF73EFF49
:101D5000002E40CF06D0DFF8FC0506431E4300F0FE
:101D60007DFB0FBDF643FFF731FF002E40CF06D0BD
:101D7000DFF8E40506431E4300F070FB0FBDF64399
:101D80000BE0E21D00000000096D6F76776D6F7645
:101D9000742C0FB5330040CF1B02300040CFFFF74B
:101DA00083FF4FF6FF7110EA014001D0FFF798FF63
:101DB0000FBD0FB50136300040CF0023FFF774FF91
:101DC000FFF78EFF06E00FB5013647F8046D0026D9
:101DD000FFF7B0FF47F8046D44F2807600F014FB83
:101DE0000FBD481E000000000563616C6C2C0FB530
:101DF000330000F086FE300040CF1B1A043BDFF8B2
:101E00005C151940002906D0DFF85425914202D014
:101E1000BDE80F40D7E740CF5B08DFF8480540F248
:101E2000FF7119400843DB0A40F2FF3119400904F1
:101E300008439B0A13F001018906084347F8046D23
:101E4000060000F00BFB0FBD7E1E00000000086CBA
:101E500069746572616C2C0008B547F8046D4FF623
:101E6000470600F0D1FA47F8046D46F6045600F034
:101E7000CBFA47F8046D0626FFF75CFF08BDA21EEB
:101E800000000000066372656174650000B500F033
:101E90003DF841F6BF60804747F8046DBEF101068A
:101EA00000BDFE1E0000200005646F65733E41F614
:101EB000BF60804747F8046DBEF10106704747F8E0
:101EC000046DBEF101064FF000521368DFF898145C
:101ED00009684FF00050834205D20F2008400428C3
:101EE00005D00231F9E70220084000D0023102316A
:101EF0001160FFF75EFF136000F0D1F900BD681FAD
:101F000000000000073C6275696C647300B500F066
:101F10009DFB4FF0005001684FF0005291420CD2EF
:101F200000F0EFFD0F200640042E40CF10D047F800
:101F3000046D362600F068FAF2E700F0E2FD0220B8
:101F4000064040CF04D047F8046D362600F05CFA16
:101F500047F8046D4BF2005600F056FA47F8046D4E
:101F60000A2600F0BEFA00BD741F00005000035B9B
:101F7000275D03E08C1F00000000012700B501F081
:101F800070F800F05EFD300040CF00BDCA1F0000B9
:101F9000300008706F7374706F6E650000B5FFF7E6
:101FA000EDFF102101400DD12021014005D0FFF7A8
:101FB00053FF47F8046DED4E04E0FFF74DFF47F87F
:101FC000046DEB4EFFF713FF00BD20200000000062
:101FD00007696E6C696E652C00B54BF200514BF6CB
:101FE000005244F270733088884208D0904208D082
:101FF000984206D047F8046D060000F005FA023654
:10200000F1E740CF00BD0EB44BF6005244F27073BE
:1020100001880230914201D09942F9D10EBC70473B
:10202000362000000000047265742C0047F8046D2F
:102030004BF60056E8E14420000030000465786962
:102040007400F3E75C20000030000772656375726E
:10205000736547F8046DC44E3668C8E67420000006
:10206000810005737461746547F8046DC14E704753
:1020700000000000862000000000015DBD48002136
:10208000C94301607047962000001000015BB94809
:10209000002101607047BE2000000000013A00B539
:1020A000B548076000F0D2FA47F8046D4BF20056CD
:1020B00000F0AAF9AF480021C943016000BD122118
:1020C00000003000013B00B5AB480168B94214D0B4
:1020D000AA498E4202D1AA4EFFF75EFCFFF714FC1C
:1020E0001520537461636B206E6F742062616C61A4
:1020F0006E6365642E0A01F040BB47F8046D4BF631
:10210000005600F081F900F0CAF89A4800210160F9
:1021100000BD2621000000000765786563757465C1
:10212000300040CF87463E210000100009696D6DE8
:1021300065646961746547F8046D1026E8E0542110
:102140000000500006696E6C696E650047F8046D0A
:102150002026DDE06E21000010000B636F6D7069BA
:102160006C656F6E6C7947F8046D3026D0E088217D
:10217000000050000A302D666F6C6461626C65006F
:1021800047F8046D4026C3E0A221000050000A3148
:102190002D666F6C6461626C650047F8046D4126C2
:1021A000B6E0BC21000050000A322D666F6C6461FD
:1021B000626C650047F8046D4226A9E0D621000054
:1021C00050000A332D666F6C6461626C650047F8DD
:1021D000046D43269CE0F021000050000A342D6677
:1021E0006F6C6461626C650047F8046D44268FE093
:1021F0000A22000050000A352D666F6C6461626C23
:10220000650047F8046D452682E024220000500056
:102210000A362D666F6C6461626C650047F8046D68
:10222000462675E03E22000050000A372D666F6C8E
:102230006461626C650047F8046D472668E06E22B1
:102240000000000008636F6E7374616E740000B567
:1022500000F0FCF9FFF700FE47F8046D44F27076D9
:1022600000F0D2F8FFF78CFF00F019F800BD9022C3
:10227000000000000932636F6E7374616E7400B504
:1022800000F0E4F939683E600E46FFF7E5FDE1E74E
:1022900000230000000006736D756467650000B5DB
:1022A0004FF0005001684FF00052914221D20239A4
:1022B0000A884FF6FF739A4205D147F8046D4FF034
:1022C000000600F0A1F800F075F800F089F82D483C
:1022D000006847F8046D06002B49096804314FF087
:1022E00000521368116000F08FF81360FEF7D7FFFB
:1022F00000BD00F05FF847F8046D4FF0000608E0FD
:102300008C230000000008736574666C61677300BD
:1023100000B54FF0005001684FF00052914205D2D5
:10232000184801683143016040CF00BD320040CF02
:1023300015480068043001884FF6FF73994201D1B7
:10234000110000E01143018000BD0000000040F2D8
:102350000000C0F200005FF000007FF00100C0FF4D
:102360000000C0FF00F800F014000020D81F00009B
:10237000EE1D0000D8FF0320100000208519120474
:102380003A1A00002000002004000020A8230000CA
:10239000410007616C69676E656401203040361842
:1023A0000220304036187047D0230000000005613D
:1023B0006C69676E00B54FF0005001680220014063
:1023C00005D047F8046D4FF0000600F01DF800BD81
:1023D000FE230000000008616C69676E31362C0036
:1023E00000B54FF0005001680F20014006D047F8BB
:1023F000046D4FF0000600F007F8F2E700BD382446
:102400000000000002682C000FB5B6B24FF000507B
:1024100001684FF00052914205D247F8046D0E005A
:10242000FEF7C7FE02E0320040CF0A8047F8046D95
:10243000022600F056F80FBD522400000000012CC7
:1024400000B547F8046DFFF7DFFF360CFFF7DCFF40
:1024500000BD6E2400000000033E3C2C00B547F890
:10246000046D360CFFF7D0FFFFF7CEFF00BDD6247A
:102470000000000007737472696E672C07B5FF21B6
:10248000314040CF300040CF002905D147F8046DDE
:102490000026FFF7B9FF07BD47F8046D067836023E
:1024A0000E43FFF7B1FF0130013902290AD347F883
:1024B000046D4678360202781643FFF7A5FF023016
:1024C0000239F2E7002900D107BD47F8046D06780C
:1024D000FFF79AFF07BD36250000000005616C6C10
:1024E0006F744FF0005001684FF00052914210D2CB
:1024F000320040CF89184FF48012914219D3FFF770
:1025000003FA0B466C6173682066756C6C0A01F007
:1025100034B9320040CF8918424A1268914208D338
:10252000FFF7F2F90952616D2066756C6C0A01F0D3
:1025300024B9016070475C250000000009666F72D5
:1025400067657472616D00B500F028F84FF00050B7
:102550003549016035483649016000BD88250000D5
:1025600000000D636F6D70696C65746F72616D3F13
:1025700047F8046D00264FF0005000684FF00051FE
:1025800088424DD3F6437047AC25000000000C6331
:102590006F6D70696C65746F72616D004FF0005003
:1025A00000684FF00051884213D370473C2600006A
:1025B00000000E636F6D70696C65746F666C61739B
:1025C00068004FF0005000684FF00051884200D280
:1025D00070471648174902680B680A6003604FF09D
:1025E0000050154902680B680A6003600D480068D6
:1025F000834215D300B5FFF787F92320566172692E
:1026000061626C657320636F6C6C696465207769C7
:1026100074682064696374696F6E6172790A00BDC1
:102620007047000024000020D40600200400002091
:10263000880100001C000020180000204627000030
:1026400000000828637265617465290000B500F018
:1026500008FD002E0ED1FFF757F915204372656172
:102660007465206E65656473206E616D6520210A56
:1026700001F083B8386847F8046D043F386000F013
:10268000AFF940CF002E40CF11D0386847F8046D25
:10269000043F3860FFF738F9095265646566696E72
:1026A0006520FFF785F9FFF72FF9022E2000FFF7CD
:1026B00081FE4FF0005000684FF00051884228D250
:1026C00095484FF000010160FFF78AFE47F8046D5E
:1026D0000C26FFF706FF00F014FA47F8046D0626F3
:1026E000FFF7FFFEFEF7DCF8FFF7C8FE8B48016836
:1026F0000A684FF0FF339A4208D14FF00052136836
:10270000116047F8046DFFF79BFE1360066040CF31
:1027100013E000F0F6F9814847F8046D0668FFF70A
:102720008FFE47F8046D4FF6FF76FFF76DFE7B488E
:10273000310040CF0160FFF7A1FE4FF0005001686B
:102740007748016000BD5E270000000008766172D6
:102750006961626C650047F8046D012613E0762715
:102760000000000009327661726961626C6547F8A9
:10277000046D022607E0542800000000096E76610F
:10278000726961626C6500B5FFF760FF4FF0005041
:1027900001684FF00052914234D20F200640B2003F
:1027A00060480168891A604A91420BD2FFF7ACF881
:1027B0000F4E6F7420656E6F7567682052414D0A29
:1027C00000F0DBBF016047F8046D0E00FFF744FB2B
:1027D00047F8046D44F27076FFF716FE300040CFE4
:1027E0000200002805D00E600431FFF729FE0138F1
:1027F000F9D147F8046D80261643FFF789FDFFF7EE
:102800004EFD00BD00F07DF90220064040CF04D10E
:1028100047F8046D3626FFF7F7FD47F8046D434E81
:10282000FFF71CFE47F8046D414EFFF717FE47F80F
:10283000046D44F27076FFF7E7FD300040CF0028CA
:1028400003D0FFF7FDFD0138FBD1FFF799FCFFF73F
:1028500026FD00BD3429000000000762756666652C
:10286000723A00B5FFF7F2FE012030403618022020
:10287000304036184FF0005001684FF0005291423E
:1028800028D228480168891B274A91420BD2FFF7BA
:102890003BF80F4E6F7420656E6F7567682052416C
:1028A0004D0A00F06ABF016047F8046D0E00FFF7A3
:1028B000D3FA47F8046D44F27076FFF7A5FDFFF7F1
:1028C000BFFD47F8046D40F24016FFF721FDFFF70A
:1028D000E6FC00BD00F015F90220064040CF04D10F
:1028E00047F8046D3626FFF78FFD47F8046D0F4E4D
:1028F000FFF7B4FD47F8046D0D4EFFF7AFFD47F845
:10290000046D44F27076FFF77FFDFFF7EAFDFFF7F5
:1029100037FCFFF7C4FC00BD2000002004000020AD
:102920001400002024000020D40600203E60043F54
:1029300002367E466629000000000F6469637469F0
:102940006F6E61727973746172744FF00050006839
:102950004FF0005147F8046D884201D2EA4E7047AB
:10296000EA4E36687047A229000000000E646963D1
:1029700074696F6E6172796E6578740003B5316841
:102980004FF0FF30814207D08879FF2804D00E0035
:1029900047F8046D002603BD47F8046D0026F64392
:1029A00003BDD429000000000A736B697073747250
:1029B000696E67003178013101220A408918761862
:1029C000704706B40178013101220A408918401885
:1029D00006BC70475C2A000000000466696E640053
:1029E00030B500220023350040CF340040CFFFF740
:1029F000ACFF4FF6FF70B188884218D047F8046DDD
:102A00000636FEF7BDFF47F8046D260047F8046D53
:102A10002E00FEF7F2FE002E40CF08D0B01DFFF7CB
:102A2000D0FF02000B004FF00050824204D2FFF7AB
:102A3000A5FF300040CFDCD0160047F8046D1E0023
:102A400030BD00B53100386803B4FFF7C9FF03BCDF
:102A50003A68002A01D100F05BFD00BDBC2A0000ED
:102A6000000006636A756D702C00320040CF3100A3
:102A700040CF8B1B043B6FF0FE01194000290ED0A4
:102A80006FF0FF0081420AD0FEF73EFF0D4A756DE0
:102A90007020746F6F206661720A00F06EBE5B106A
:102AA000FF210B40134330001E0000B54FF00052D1
:102AB00013681060FFF7A8FC136000BDF62A000041
:102AC0000000056A756D702C310040CF300040CF9A
:102AD0000B1A043B8E491940002902D08D4A9142BD
:102AE000D2D15B1040F2FF72134053F4604347F8B9
:102AF000046D1E00D9E70E2B00000000046865720B
:102B0000650047F8046D4FF00056366870470A2C90
:102B1000000000000D666C6173687661722D686557
:102B2000726547F8046D7C4E3668704700B547F80B
:102B3000046D42F60066FFF767FC47F8046D4CF63B
:102B40004076FFF761FC00BDDBE700B500F03AF826
:102B500039683E600E4647F8046D4DF20016FFF7E7
:102B600084FF00BD00B500F02DF839683E600E46C8
:102B700047F8046D4DF20076FFF777FF00BD00B512
:102B8000FFF7D4FF00F01EF839683E600E4647F8A4
:102B9000046D4DF20006FFF768FF00BD00B500F0C0
:102BA00011F839683E600E46FFF78EFF00BD00B594
:102BB000FFF7BCFFFFF7A5FF47F8046D0226FFF7FC
:102BC00090FC00BD00B5FFF79CFF47F8046D02269E
:102BD000FFF787FC00BD00B5FFF793FFFFF774FF19
:102BE00000BD00B5FFF78DFF47F8046D4DF20006FC
:102BF000FFF73BFF00BD00B5FFF783FF47F8046D0B
:102C00004DF20016FFF731FF00BD462C00003000EA
:102C1000047468656E00052E01D140CFDBE7022EFB
:102C200001D140CFDDE7FEF76FFE17537472756375
:102C3000747572657320646F6E2774206D617463A0
:102C4000680A00F09ABD622C0000300004656C73C5
:102C5000650000B500F017F8FDF7C4FAFFF7DBFFD9
:102C600000BD7A2C000030000269660000B5FFF755
:102C70009EFF47F8046D022600BD942C0000300032
:102C800005616865616400B5FFF79CFF47F8046D56
:102C9000052600BDAE2C000030000672657065612F
:102CA000740000B500F01FF8FFF7B5FF00BDC62C9B
:102CB00000003000057768696C6500B5FFF7D6FF46
:102CC000FDF790FA00BDDA2C0000300005756E7437
:102CD000696C012EA7D140CF51E7EE2C00003000E7
:102CE00005616761696E012E9DD140CF56E71C2DAD
:102CF0000000300005626567696E00B5FFF724FFCC
:102D000047F8046D012600BD880100000400002082
:102D100001F8FFFF00F8FFFF240000202C2D000029
:102D20002000016B47F8046D029E70473C2D0000A7
:102D30002000016A47F8046D009E70474C2D00008A
:102D40002000016947F8046D260070478A2D0000B5
:102D50003000056C6561766500B5D84801683B00B8
:102D6000043F1A68043B1A6008338B42F9D103B45C
:102D7000FFF728FF03BC330040CF04390B6001602C
:102D800004390A6801320A6000BD9C2D0000200051
:102D900006756E6C6F6F700030BC7047D42D0000EC
:102DA0003000052B6C6F6F70032E00D03BE740CFD7
:102DB00000B547F8046DC24EFFF70EF9FFF7D2FEDB
:102DC0001AE014F10044641BA41940CF2C44A4F170
:102DD00000447047162E00003000046C6F6F7000C6
:102DE000032E00D01FE740CF00B547F8046DB54E65
:102DF000FFF7F2F8FFF7A9FE00F019F9AF4831002C
:102E000040CF016047F8046DAF4EFFF7E5F800BD15
:102E10000134AC4270475E2E0000780002646F00FF
:102E200000B547F8046DA94EFFF7D6F8A34801682E
:102E300047F8046D0E0047F8046D00260760FFF7A1
:102E400083FE47F8046D032600BD00B500F02FF89F
:102E5000ECE730B4340040CF350040CF7047F82E57
:102E600000007800033F646F00B547F8046D974E8B
:102E7000FFF7B2F847F8046D44F2AC26FFF7C4FA46
:102E80008E48016847F8046D0E00FFF79BFE01367F
:102E900047F8046D012689480760FFF755FE47F89B
:102EA000046D032600BD00B500F001F8E2E700B5AF
:102EB00047F8046D4BF23046FFF7A6FA47F8046D69
:102EC0000426FEF737FF013B08D047F8046D0526BE
:102ED000FEF730FF013B00F029FC00BD47F8046D10
:102EE0003526FFF791FA47F8046D4CF64076FFF768
:102EF0008BFA00F01BFC00BD122F000030000463B1
:102F00006173650047F8046D002647F8046D0826D4
:102F10007047282F00003000033F6F666C4809E0BF
:102F2000013EB64140CF7047CE2F00007800026FBF
:102F300066006848082E00D075E640CF00B547F817
:102F4000046D0600FFF748F8FFF73CFE39683E6065
:102F50000E46013647F8046D092647F8046D4CF615
:102F60004076FFF751FA00BD00B5300040CF013B7D
:102F700001B400F0DBFB01BC082E00D053E640CFCB
:102F800047F8046D0600FF213140B14205D14FF4EE
:102F900038510E43FFF738FAD6E7FEF717FE002E3A
:102FA00040CF04D04C480643FFF758FACCE747F827
:102FB000046D0026FEF7BEFE47F8046D44F2B0260D
:102FC000FFF722FAC0E7300040CFB042704704302C
:102FD0000000300005656E646F66092E00D022E6A1
:102FE00040CF00B540B440CFFFF7ECFD39683E60FC
:102FF0000E46FFF700FE47F8046D40BC47F8046D2D
:10300000082600BD56300000300007656E6463611D
:103010007365082E00D006E640CF00B547F8046D72
:103020004CF64076FFF7F0F900F001F800BD00B56E
:10303000300040CF00280DD003B4012131400029D9
:1030400003D0013EFFF7CDFD01E0FFF7C4FD03BC57
:103050000138EFE700BD6A300000000005746F6BB7
:10306000656E47F8046D202605E0E430000000009E
:1030700005706172736510B5184801684068184A98
:1030800012688418202E07D191420FD0835CB3427E
:1030900002D101328418F7E7914207D0835C0132F4
:1030A000B342F9D18618361B013E01E08618361B63
:1030B000043F3C600A48026010BD00000C00002084
:1030C000C22D0000102E0000982D0000522E00008E
:1030D000202F0000C62F0000000FB6F1DCFF0320F8
:1030E000E4FF032022310000000005646967697471
:1030F000CF4B1B68303E0BD30A2E0BD3073E0A2E54
:1031000006D3242E06D3203E0A2E01D3242E01D32B
:10311000002670479E42FBD247F8046D0026F64316
:1031200070472C3200000000066E756D62657200FB
:103130003FB5310040CF701E0126012204B4BC4BC4
:103140001B680024002500293CD001300139027899
:103150002D2A04D101B00022D24304B4F3E7232A7C
:1031600001D10A23EFE7242A01D11023EBE7252A16
:1031700001D10223E7E72E2A01D10226E3E72C2A18
:1031800036D047F8046D1600FFF7B4FF002E40CF8D
:103190002BD047F8046D260047F8046D2E0047F841
:1031A000046D1E0047F8046D00260FB4FDF718F9F2
:1031B0000FBC350040CF340040CF0022A419554148
:1031C00040CFC0E704BC002A04D50022E443ED430D
:1031D0000134554133002600012B02D047F8046D1D
:1031E0002E0047F8046D1E003FBD01B000263FBD14
:1031F0002500002402260029E4D0425C01392E2A51
:10320000F9D047F8046D1600FFF774FF002E40CF89
:10321000EBD0043F3C6047F8046D1E000FB4FDF78F
:103220008EF90FBC340040CF40CFE4E74E320000AF
:103230000000062E6469676974000A2E01D23036D8
:103240007047242E01D237367047232670478432C8
:103250000000000004686F6C6400330040CF7548C4
:1032600001783F290DD2013101704018012907D0A2
:103270000138027801300270013801390129F7D193
:1032800003707047A4320000000005686F6C643C56
:10329000330040CF674801783F2902D201310170E5
:1032A00043547047BC3200000000047369676E002D
:1032B000002E01D440CF70472D26CEE7D03200003B
:1032C000000002233E005B480678013038607047FA
:1032D000E832000000000366235310B5202400F0FC
:1032E00008F8013CFBD110BD0A3300000000026663
:1032F000230000B547F8046D4D4E3668FDF75CF8C5
:10330000FFF79BFFFFF7C4FF00BD2633000000005E
:103310000223530000B500F00AF8002EFBD13868F4
:103320000028F8D100BD523300000000012300B591
:1033300047F8046D3E4E366847F8046D0026FDF7E9
:103340001DF9FCF74FFF40CFFFF777FFFFF785FF31
:1033500000BD643300000000023C2300354800211A
:103360000170704776330000000002662E0047F8B7
:10337000046D202604E0C4330000000003662E6EB6
:1033800000B510B4340040CFFDF774FAFCF7DDFF50
:1033900047F8046D0026FFF7E1FFFFF7BBFF40CFC2
:1033A0002C26FFF775FF002C03D0FFF7A2FF013C8E
:1033B000FBD110BC40CFFFF77BFF47F8046D47F807
:1033C000046D1CE0DA33000000000375642E00B5C4
:1033D000FFF7C4FFFFF79EFF11E00C340000000070
:1033E00002642E0000B5FDF745FAFCF7AEFFFFF7CB
:1033F000B5FFFFF78FFFFDF747FAFFF759FFFFF71C
:1034000062FFFEF7D5FAFEF72EFA00BD1E3400006B
:10341000000002752E0047F8046D0026D7E7383407
:1034200000000000012E47F8046DF617DAE70000EF
:10343000FCFF032028000020803400000000086505
:1034400076616C756174650000B5FEF7AAF901CF6D
:1034500001B440B440CFD948016802B400210160F2
:10346000FEF792F900F014F8D44802BC016047F866
:10347000046D40BC01BC043F3860FEF785F900BD17
:1034800052370000000009696E74657270726574CD
:1034900030B5CB4887420BD9FEF736FA105374612A
:1034A000636B20756E646572666C6F770A0064E109
:1034B000C44887420AD2FEF727FA0F537461636B40
:1034C000206F766572666C6F770A56E1BE4C256890
:1034D000002D01D13D002560FFF7C3FD002E02D174
:1034E000043740CF30BD386847F8046D043F38607A
:1034F000FFF776FA310040CF320040CF002A19D1D1
:1035000038683100FFF714FE320040CF002AC0D1E6
:1035100047F8046D060047F8046D0E00FEF748FA00
:10352000FEF7F2F90C206E6F7420666F756E642ED4
:103530000A0022E1A54B1B68002B1DD10025256048
:1035400030230B40302B0ED1FEF732FAFEF7DCF9B8
:103550001220697320636F6D70696C652D6F6E6CDE
:10356000792E0A0009E1043740CF47F8046D1600B0
:10357000FEF7D6FDFFF78DFF043740CF80200840CF
:103580000ED1EB1B9B08402008400FD008200840BC
:1035900002D0002B00D01DE00F200840834205D34D
:1035A00047F8046D1600FEF7BBFD72E700F0BEF8A9
:1035B00047F8046D160010220A4002D0FEF7B0FD55
:1035C00067E720220A4002D0FEF706FD61E7FEF71A
:1035D0000EFC5EE7072001401000FEF714FD0129F4
:1035E0001FD1012BDCD1FF213140B14204D14088F1
:1035F0000643FEF709FF4CE7FEF7E8FA002E40CF3E
:1036000004D040680643FEF729FF42E747F8046DFF
:103610000026FEF78FFB47F8046D0688FEF7F4FEE0
:1036200037E7022902D1012BBAD1EFE7032927D1CD
:10363000012BB5D1FF213140B1420BD14FF478516C
:103640000E43FEF7E1FE043247F8046D1600FEF764
:10365000C3FC1EE7FEF7BAFA002E40CF04D05C4947
:103660000E43FEF7FBFEEEE747F8046D0026FEF77B
:1036700061FB023247F8046D1600FEF7ADFC08E767
:10368000042918D1012B8BD1330040CF002B00D15E
:10369000FFE61F221A409A4205D047F8046D46887B
:1036A000FEF7B2FEF5E647F8046D06889B011E435F
:1036B000FEF7AAFEEDE6052924D1012B10D147F82B
:1036C000046D0026FEF736FB47F8046D0600FEF792
:1036D00083FC47F8046D4CF64076FEF795FED8E67D
:1036E00047F8046D0026FEF725FB47F8046D012618
:1036F000FEF720FBFEF787FC47F8046D0600FEF797
:103700006BFCC6E606290ED1012B7FF449AFFEF70C
:103710005DFA002E40CF3FF479AFD0F802000643A7
:10372000FEF79CFEB5E601308047B2E600B5002BFF
:103730000CD0013B47F8046D1E0057F82660FEF7D9
:103740008BFB002BF5D1043D2F0040CF00252560D9
:1037500000BD6E370000810009686F6F6B2D7175B9
:10376000697447F8046D1B4E7047A6370000E837B0
:1037700000000000047175697400DFF85CD0104F20
:10378000FDF707FD15480A2101601048002101607E
:103790000D4801600948016011480160114941600C
:1037A0000C4800688746FEF70AF8FFF771FEFEF73F
:1037B000ABF805206F6B2E0AF5E70000E4FF03204D
:1037C000300300203001002008000020D8FF032033
:1037D0000006B6F1D4FF032030040020FCFF0320D4
:1037E000DCFF0320680000200238000000000565AF
:1037F000696E743F47F8046DEFF31086013EB641E1
:1038000070471238000020000465696E740062B6CB
:1038100070472238000020000464696E740072B69C
:10382000704738380000200004697073720047F850
:10383000046DEFF305867047443800000000036E06
:103840006F70704786380000000009756E68616E01
:10385000646C656400B5FEF757F814556E68616EC8
:10386000646C656420496E746572727570742000B2
:1038700047F8046DEFF30586FEF7AEF8FEF744F85F
:1038800002210A0000BD983800000000057265732F
:103890006574C848C8490160C238000081000B69DE
:1038A00072712D7379737469636B47F8046DC34E3D
:1038B0007047543800004FF6D070C2F20300006821
:1038C0008746EA3800008100096972712D666175CA
:1038D0006C7447F8046DBA4E7047543800004FF6C8
:1038E000CC70C2F2030000688746183900008100DE
:1038F0000E6972712D636F6C6C656374696F6E0015
:1039000047F8046DAF4E7047543800004FF6C8704A
:10391000C2F203000068874640390000810009694F
:1039200072712D657874693047F8046DA64E704742
:10393000543800004FF6C470C2F203000068874696
:10394000683900008100096972712D6578746931E8
:1039500047F8046D9D4E7047543800004FF6C07014
:10396000C2F20300006887469039000081000969AF
:1039700072712D657874693247F8046D944E704702
:10398000543800004FF6BC70C2F20300006887464E
:10399000B83900008100096972712D657874693346
:1039A00047F8046D8B4E7047543800004FF6B870DE
:1039B000C2F2030000688746E0390000810009690F
:1039C00072712D657874693447F8046D824E7047C2
:1039D000543800004FF6B470C2F203000068874606
:1039E000063A00008100076972712D61646347F82F
:1039F000046D7A4E7047543800004FF6B070C2F232
:103A00000300006887462E3A000081000869727141
:103A10002D74696D320047F8046D714E704754384B
:103A200000004FF6AC70C2F2030000688746563AB9
:103A300000008100086972712D74696D330047F8C8
:103A4000046D684E7047543800004FF6A870C2F2FB
:103A50000300006887467E3A0000810008697271A1
:103A60002D74696D340047F8046D5F4E704754380B
:103A700000004FF6A470C2F20300006887460C40B5
:103A80000000FFFF182D2D2D20466C617368204427
:103A9000696374696F6E617279202D2D2D00FDF7B9
:103AA000E2FC52488546524F2A264FF000505149B9
:103AB000016051485149016047F8046D4F4E504D27
:103AC000B1884FF6FF73994225D04FF480730B40B5
:103AD0000AD0B01DFEF775FFFEF795FA03884088FF
:103AE00000040343ED1A16E080230B4013D00F238C
:103AF000194089006D1AB01DFEF763FFFEF783FAC7
:103B000047F8046D060047F8046D2E0047F8046D71
:103B10000E00FDF75DF8FEF731FF300040CFCFD04B
:103B20003848066040CF384805604FF480104FF4A5
:103B300080414FF6FF72884204D0023803889342D6
:103B4000F9D0023031490860FDF723FBFDF7DCFEB8
:103B5000384D6563726973702D5374656C6C617256
:103B6000697320322E352E3220666F722053544DE9
:103B7000333257423535206279204D61747468695B
:103B80006173204B6F6368200A00214800210160A7
:103B900047F8046D1F4E47F8046D0426FEF720FF1A
:103BA00040CF002E02D0FEF7BBFAF9E540CFE4E5A6
:103BB000696E69740CED00E00400FA05D0FF032083
:103BC000CCFF0320C8FF0320C4FF0320C0FF032055
:103BD000BCFF0320B8FF0320B4FF0320B0FF032085
:103BE000ACFF0320A8FF0320A4FF03203004002023
:103BF00030030020D40600200400002088010000CB
:103C0000000004201C0000202400002018000020D8
:083C100008000020B03B000099
:0400000508000000EF
:00000001FF
